:100000000C94AC020C94E4020C94E4020C94E40210
:100010000C94E4020C94E4020C94E4020C94E402C8
:100020000C94E4020C94E4020C94E4020C948F1EF1
:100030000C943E1F0C9458190C94E4020C94E402A6
:100040000C94E4020C94E4020C94E4020C94E11984
:100050000C94E4020C94E4020C94E4020C94E40288
:100060000C94E4020C94E4020C94E4020C94E40278
:100070000C94E402530553057F057F05E005D70680
:10008000D706D706FE056606770677064E14C01417
:100090005614201424145A1427145D1468143214AE
:1000A000B61436146C143A1470149A143E14741462
:1000B000A41444147A1484142B1461142E1464149C
:1000C00049147F149014B014B2141C145214C9149F
:1000D0007B1681166F16751687168D169316901758
:1000E0009317CA17DD17E517F017F317F317F31770
:1000F0003B183B18F817FB1700180D181A181D1895
:1001000021182E18A61FCD1FC520CD1FC5201920D0
:100110003C20C5209320A22029001E001F002000A3
:1001200021002200230024002500260027002D00A6
:100130002E0000002A002B0014001A0008001500F1
:1001400017001C0018000C00120013002F003000D4
:1001500031000000E00004001600070009000A005A
:100160000B000D000E000F003300340028000000CB
:100170000000E10000001D001B0006001900050042
:1001800011001000360037003800E50000000000C4
:10019000E000E300E2002C002C002C00E600E70069
:1001A0006500215200000000000000000000007CFB
:1001B0003A003B003C003D003E003F004000410053
:1001C000420043004400450001000100010001001D
:1001D00052000100010001000100010001000100C6
:1001E0000100010001000100000001005000510069
:1001F0004F000100010001000100010001000100A9
:1002000001000100000000000100010001000100E8
:1002100001000100010001000100010001000100D6
:1002200001000100000001000100010001000100C7
:1002300001000100010001000100000000000000B9
:1002400000000000010001000100010001000100A8
:100250000100010001000100010001000100010096
:100260000100010001000100010001000100010086
:100270000100010001000100010001000100000077
:100280000100010001000100010001000100010066
:100290000100010001000100010000000000010058
:1002A0000100010001000100010001000100010046
:1002B0000100010001000100010000000100010037
:1002C0000100010001000100010001000100010026
:1002D000000000000000000000000100010001001B
:1002E0000100010001000100010001000100010006
:1002F00001000100010001000100010001000100F6
:1003000001000100010001000100010001000100E5
:1003100001000100000001000100010001000100D6
:1003200001000100010001000100010001000100C5
:1003300000000000010001000100010001000100B7
:1003400001000100010001000100010001000100A5
:100350000000010001000100010001000100010096
:10036000010001000100000000000000000000008A
:1003700000000000000000002A2B28000000000000
:100380000000000000000000000000290000000044
:100390002C1E3420212224342627252E362D3738B2
:1003A000271E1F202122232425263333362E3738BB
:1003B0001F0405060708090A0B0C0D0E0F10111279
:1003C000131415161718191A1B1C1D2F3130232D45
:1003D000350405060708090A0B0C0D0E0F10111243
:1003E000131415161718191A1B1C1D2F3130354CF4
:1003F00000000000000000000000000000000000FD
:1004000000000000000000000000000000000000EC
:10041000000000007E0F00D4FFFFFFC7000000783F
:100420001C0362006F006F0074006C0065006700C1
:1004300020005200650076002000410000000E03FD
:100440003400700070006C0065007400000004034C
:10045000090409025B00030100A0FA09040000017D
:100460000301010009211101000122440007058157
:100470000308000109040100020300000009211122
:100480000100012222000705820320000107050365
:1004900003200001090402000103000000092111EA
:1004A000010001223200070584032000011201002F
:1004B000020000000844440400010001020001069B
:1004C00060FF0961A1010962150026FF00952075F2
:1004D0000881020963150026FF0095207508910226
:1004E000C005010980A101850319012AB700150182
:1004F00026B700950175108100C0050C0901A10106
:10050000850419012AA002150126A0029501751083
:100510008100C005010906A101050719E029E715B9
:100520000025019508750181029501750881010575
:1005300007190029FF150026FF00950675088100A0
:100540000508190129051500250195057501910278
:10055000950175039101C00011241FBECFEFD4E0B7
:10056000DEBFCDBF04B603FE18C080917902909122
:100570007A02A0917B02B0917C028730904BA74019
:10058000B04B59F41092790210927A0210927B02C9
:1005900010927C02E0E0F8E3099511E0A0E0B1E000
:1005A000E4E6F3E402C005900D92A63AB107D9F74C
:1005B00022E0A6EAB1E001C01D92A937B207E1F737
:1005C0000E94F4110C94B0210C940000282F843068
:1005D000E8F46530D8F44F30C8F4862F90E06FE02F
:1005E00070E00E94F320FC01822F90E06BE470E049
:1005F0000E94F3208E0F9F1FFC01E40FF11DEE0FF0
:10060000FF1FE85EFE4F85919491089581E090E090
:10061000089581E0089581E008950E940B030895F4
:100620000E940D0308950E940B03089508950E94EF
:1006300016030895A6E0B0E0E0E2F3E00C94202178
:1006400049835A839E833091AD0189819A8131110A
:1006500015C03E81332359F0222349F00E947108CE
:10066000182F682F89819A810E94480803C00E9430
:100670005D08182F69817A81812F04C00E9471085A
:1006800069817A810E94A70F2696E3E00C943C21B1
:10069000FC01262F40815181628173818481958183
:1006A0000E941A030895CF93DF93EC0161E00E944A
:1006B0004803BE010E941003DF91CF910895CF93AC
:1006C000DF93EC0160E00E944803BE010E94170323
:1006D000DF91CF91089581E008950E946B03089502
:1006E000CF93C82F0E9444078C2F0E946D032FEFD9
:1006F00084E39CE0215080409040E1F700C000007E
:10070000CF91089581E00E9470030E94071A089516
:1007100080E00E9470030E942B1A08950F931F938C
:10072000CF93DF938C0161E00E944803EC01B80194
:100730000E945D17882309F450C0B801CE010E94C1
:100740001303882309F449C0B801CE010E9463163F
:10075000882309F442C0B801CE010E94F81388230F
:10076000E1F1B801CE010E94CE138823B1F1B801A6
:10077000CE010E94A616882381F1F8018581882385
:1007800041F1C3308CE7D807D1F040F4C115FCE744
:10079000DF0791F0C130DC47A1F01BC0CB35ECE79F
:1007A000DE07A9F0CC35FCE7DF0771F0CA35DC477E
:1007B00081F40E94D10C0DC00E9482030EC00E94E1
:1007C000D90C0E94880309C00E94C70C02C00E9475
:1007D000D50CC8010E94090301C080E0DF91CF91D0
:1007E0001F910F9108950E9436190E941A040895CE
:1007F0000E941E040E943F190895089581E0089503
:100800000895CF93DF93D82F0E94FE03C82F88232B
:1008100019F08D2F0E9400048C2FDF91CF91089545
:100820000895CF93C82F0E94FD038C2F0E940104CE
:10083000CF91089580E00E94110408950E944B1802
:100840000E9411040895CF930E944B18C82F8091E5
:10085000A801C81779F0C093A8010E94C619609337
:10086000A9017093AA018093AB019093AC018C2FE6
:100870000E941104CF910895ADE0B0E0E2E4F4E00D
:100880000C942121488759876A877B878C879D87AD
:1008900091110E94030CCE01019627E0FC011192F8
:1008A0002A95E9F726E0FE013896DC0101900D92C9
:1008B0002A95E1F72D8121110AC029813A814B81C6
:1008C0005C816D817E818F810E94440B04C00E94F7
:1008D00053038111F2CF2D96E2E00C943D21FC01EF
:1008E0002481213021F4808191810E949E08089505
:1008F000CF938823D9F1C82F8CEF8C0F813A70F4F5
:100900008C2F0E94BC18882329F08C2F0E94FF187E
:100910000E94650C8C2F0E94F7180CC080E28C0F8F
:10092000883058F4C77081E001C0880FCA95EAF793
:100930000E94E60B0E94650C19C0EBE5EC0FE3305A
:1009400040F4F0E0EA5BFE4F808190E00E94631883
:100950000DC0C85ACB3150F4EC2FF0E0EE0FFF1F62
:10096000E05FFE4F808191810E948818CF910895A9
:10097000882339F19CEF980F913A18F40E94FF18E0
:100980000DC090E2980F983060F4877091E001C03C
:10099000990F8A95EAF7892F0E94EC0B0E94650C4B
:1009A00008959BE5980F933028F480E090E00E9432
:1009B00063180895885A8B3120F480E090E00E94FB
:1009C000881808951F93CF93DF93182FEB010E948F
:1009D0007804209741F08FE99FE00197F1F700C07C
:1009E00000002197F6CF812F0E94B804DF91CF91AC
:1009F0001F910895893319F060E070E002C060E54E
:100A000070E00E94E2040895882321F00E94E60B22
:100A10000E94650C0895882321F00E94EC0B0E942F
:100A2000650C0895A0E0B0E0E8E1F5E00C941B212E
:100A30007C01162FC72FFC01D581068102950F700E
:100A40000E94DC0B8823F9F0DD23E9F08C2F807FF6
:100A5000803461F080E2810F8830A8F08C2F807E96
:100A6000803221F4123078F0002369F08091530233
:100A700082FF09C082E00E949B0C0E94DC0B91E087
:100A8000D82ED92601C0D12CCC2EC2948FE0C822FA
:100A90008C2D90E08C30910508F089C1FC01E65C5A
:100AA000FF4F0C9404218C2F807FCF70882311F08E
:100AB000C295C07FDD2399F0CC2309F464C180E2A4
:100AC000810F883010F0111104C08C2F0E94E60BAA
:100AD00003C08C2F0E94F60B0E94650C54C1812F1D
:100AE0000E94B804CC2309F462C180E2810F8830EF
:100AF00038F1112329F18C2F0E94FC0B24C08C2F7C
:100B0000807FCF70803211F0C295C07F112319F021
:100B1000113099F13CC08091530282FD17C0DD2352
:100B200049F0CC2329F08C2F0E94E60B0E94650C23
:100B300080E02AC180E00E94B804CC2309F437C1C8
:100B40008C2F0E94EC0B0E94650C31C1DD2349F013
:100B5000002309F1013009F02AC18C2F0E940D0CED
:100B600026C1011124C18C2F0E940B058C2F0E94DD
:100B7000190C8C2F0E946E0C1AC1DD2321F0063057
:100B800008F015C108C0053008F011C115C0DD23FB
:100B900031F00111F8C08C2F0E94040508C1002318
:100BA00059F0193309F000C1FFEF27EE83E0F1504F
:100BB00020408040E1F7F6C08C2F0E940B05F7C063
:100BC0008C2F86958695837019F0813061F0EFC087
:100BD000DD2321F0812F9C2F937002C080E090E0F4
:100BE0000E946318ECC0DD2321F0812F9C2F9370AD
:100BF00002C080E090E00E948818E1C08C2F8370D2
:100C000079F5D111D8C0412F429546954770440FD0
:100C1000440F212F2F70042E01C0220F0A94EAF7EF
:100C200014FF08C08FE090E001C0880F4A95EAF7F2
:100C3000809501C080E0C695C695C370822BC230F6
:100C400049F058F4C13019F00E949B07B4C00E94CB
:100C50009507B1C00E94A107AEC00E949207ABC029
:100C6000DD2319F08C2F817001C08695882309F44B
:100C7000A2C0412F429546954770440F440F212F43
:100C80002F70042E01C0220F0A94EAF714FF08C047
:100C90008FE090E001C0880F4A95EAF7809501C087
:100CA00080E0C695C695C370822BC23049F058F4D7
:100CB000C13019F00E94E7077EC00E94E1077BC0A7
:100CC0000E94ED0778C00E94AA0775C0CF70DD238F
:100CD00039F08C2F0E94BC07812F0E9404056BC045
:100CE000812F0E940B058C2F0E94C80764C0123F01
:100CF00021F128F4103F41F0113FC1F040C0133FF3
:100D000019F1143F79F03BC0DD2341F0053008F0C4
:100D10004EC08C2F8F710E94D50749C0063008F055
:100D200046C0F7CF8091530282FD18C0DD2339F011
:100D30008C2F8F710E94BC073AC0DD23C9F38C2F22
:100D40008F710E94C80733C0DD2329F08C2F8F716B
:100D50000E94B3072CC00E94AF0729C0DD2331F0E9
:100D600063E08C2F8F710E947D0C21C081E00E9476
:100D70009B0C0230E0F082E00E949B0C18C0DD2347
:100D800031F00023A9F2812F0E94780410C00023C3
:100D9000B1F2193349F49FEFE7EEF3E09150E040F0
:100DA000F040E1F700C00000812F0E94B80488EFF6
:100DB0008C0D843020F40E944B180E941104DD2019
:100DC00089F00E94D80B80FD0DC0F70115820E94AA
:100DD000D20B0E94BC07C7010E940F070E94D20BD2
:100DE0000E94C807CDB7DEB7E8E00C9437210F9317
:100DF0001F93CF93DF93EC01688179818D810E94ED
:100E0000A9088C010E94F3070E948507B801CE0152
:100E10000E941205DF91CF911F910F910895CF93FA
:100E2000DF93FC0124812223D1F0EC010E948E0388
:100E300081110FC00E94DC0B882389F08D818823EB
:100E400071F08091530282FF0AC082E00E949B0CE5
:100E500006C0CE010E94F706CE010E945F03DF911B
:100E6000CF91089580E090E00E94631880E090E0C8
:100E70000E9488180E94030C0E94650C08950E942D
:100E800007190E94320708950E94F30B0E943F0742
:100E9000089592959F70963079F010F4925001C0A9
:100EA0009A50923068F4803F69F018F4883E40F41C
:100EB00009C0843F29F406C0883E20F0813F11F02C
:100EC00080E0089581E00895FC012481222339F017
:100ED000808191810E949E080E944907089580E0C8
:100EE0000895A6E0B0E0E7E7F7E00C94212126960C
:100EF000E2E00C943D21A7E0B0E0E1E8F7E00C94DB
:100F000021212796E2E00C943D21089508950E9446
:100F1000860708950E94870708950E948A07809394
:100F2000CD0108950E948D0708959091CD01892BE0
:100F30000E948D0708959091CD0189230E948D070D
:100F400008959091CD0189270E948D0708950E94F0
:100F5000860708950E94A7078093CC01089580E03A
:100F60000E94AA07089591E001C0990F8A95EAF7B7
:100F7000892F0E94AA07089521E030E001C0220FC6
:100F80008A95EAF78091CC01822B0E94AA070895E6
:100F900021E030E001C0220F8A95EAF72095809188
:100FA000CC0182230E94AA07089521E030E001C00D
:100FB000220F8A95EAF78091CC0182270E94AA0726
:100FC00008959091CC01892B0E94AA0708959091D1
:100FD000CC0189230E94AA0708959091CC0189270A
:100FE0000E94AA0708950895282FFA01862F877076
:100FF000A1E001C0AA0F8A95EAF7CB0133E09695EC
:1010000087953A95E1F763E070E00E94F320E80FDE
:10101000F91F40E050E0622F70E090819B01042EA8
:1010200002C0369527950A94E2F721702195292769
:101030002A23292721934F5F5F4F4330510569F7DA
:101040000895FB01A82FA77023E0969587952A9510
:10105000E1F763E070E00E94F320E80FF91F40E041
:1010600050E080E0219130E00A2E02C036952795AD
:101070000A94E2F721703327042E01C0220F0A944C
:10108000EAF7822B4F5F5F4F4330510559F70895C0
:10109000953090F48F3080F4362F282F892F90E0F0
:1010A0006FE070E00E94F320BC01620F711D4EEAF8
:1010B00051E0832F0E94F4070895953080F48F301B
:1010C00070F4282F892F90E06FE070E00E94F320E9
:1010D0006EEA71E0820F911D0E942108089580E060
:1010E0000895CF92DF92FF920F931F93CF93DF93D8
:1010F0006C010091CC018091CD01082BC3E0D0E0C0
:1011000010E0C8010C2E02C0959587950A94E2F76D
:1011100080FD04C02197A8F7F12C07C0FC2EB60172
:101120008C2F0E94B30F0197A9F38F2DDF91CF91E0
:101130001F910F91FF90DF90CF900895CF93DF9391
:10114000EC010E947108BE010E94B30FDF91CF91A4
:1011500008951F93CF93DF93EB019091AD019923F5
:1011600021F0CB010E949E0813C0882349F0CB01D7
:101170000E947108182F682FCE010E94480804C0F1
:10118000CB010E945D08182FBE01812F0E94B30F72
:10119000DF91CF911F910895E1E0F0E0DF0102C0FF
:1011A000AA0FBB1F6A95E2F7BD01DF0102C0AA0FBB
:1011B000BB1F4A95E2F7AD01462B01C0EE0F2A9501
:1011C000EAF7942F9823491302C08E2B0895E095D7
:1011D0008E230895242F462F682F8091CC010E94E2
:1011E000CC080E94AA070895CF93DF93C091CE0147
:1011F0008091CF01C817A9F0D0E0CE0167E070E080
:101200000E94F320FC01E053FE4F20813181428196
:1012100053816481758186810E947B072196C77006
:10122000E7CFDF91CF910895209108023091090214
:1012300040910A0250910B0260910C0270910D02D4
:1012400080910E020E947B070895CF93DF938091D7
:101250000E0282958F7009F04CC080910D02882398
:1012600009F447C02091CE014091CF01A09109021D
:10127000B0910802C0910A02D0910B022417C9F163
:1012800030E0C90167E070E00E94F320FC01E05308
:10129000FE4F8481882349F181818A1326C0808191
:1012A0008B1323C08581811120C0828193818C1B87
:1012B0009D0B883C9105C8F480910E028F7080616F
:1012C00080930E02C90167E070E00E94F320FC01E8
:1012D000EA52FE4F90819F709061908388E092E087
:1012E0000E940F070E94F40804C02F5F3F4F277031
:1012F000C5CFDF91CF910895CF93B82FC62F2091FE
:10130000CE01A091CF012A17B1F030E0C90167E00A
:1013100070E00E94F320FC01E053FE4F81818C13AA
:1013200006C080818B1303C08581841306C02F5FA4
:101330003F4F2770E8CF80E001C081E0CF91089552
:10134000A4E1B0E0E6EAF9E00C9417218C0186E014
:10135000F801DE011F9601900D928A95E1F7F801E0
:101360008481E58098E0A92E92E0B92E90910C023C
:10137000911118C0882309F480C1EE20D9F1C80169
:101380000E946407F82E8823A9F187E0F801D501AF
:1013900001900D928A95E1F7C5010E946F040E94A9
:1013A000250998C0F801C080D18082809380F09098
:1013B0000D0220910A0230910B02A401421B530B33
:1013C000FF2009F406C1483C510508F0AFC088234E
:1013D00009F455C180910E02282F207F90910902B7
:1013E000222361F09D1509F462C0C8010E946407C0
:1013F000811173C0C8010E940F073FC19D1115C024
:10140000909108029C1111C0E1100FC08F70806193
:1014100080930E020E94140988E092E00E940F0758
:1014200080910E02F801868326C1E1103AC040E0A7
:101430006D2D8C2D0E947C0940E06D2D8C2D0E941D
:101440007C09E82E811117C1CF86D88A8F859889AB
:101450000E949E08292F22952F70243020F49F701F
:10146000223028F009C02A50223080F014C099237D
:1014700049F0811107C013C0992321F0F80196812A
:10148000907F69F0805E883030F409C0803F38F08A
:10149000815F833020F0C8010E940F07EF2CFE2CE3
:1014A000EEC080910E02816080930E02E4C09091A4
:1014B00008029C119ACFE11098CFF8018683C801E9
:1014C0000E940F0787E0F801A8E0B2E001900D92BA
:1014D0008A95E1F70E941409D2C0EE2009F48ACF60
:1014E00020910E02822F82958F7090E002978CF0EF
:1014F0008091080290910902998788879B868A8645
:1015000080910C028C871D862E87CE0108960E9442
:101510000F0787E0F801A8E0B2E001900D928A95EC
:10152000E1F70E9425090E941409A7C090910E02BC
:10153000292F207FA1F4682D9A8A898AA6017A89A9
:101540009E2D0E94710788E092E00E940F0787E0BD
:10155000F50111928A95E9F70E9414098CC088233D
:1015600009F48DC0809109028D1111C0809108028B
:101570008C110DC0E1100BC0F8019683C8010E94C8
:101580000F0787E0F50111928A95E9F778C0C80145
:101590000E946407882309F42DCFEE2009F42ACF96
:1015A00020910E02822F82958F7090E002970CF4AA
:1015B000B0CF80910802909109029A8389839C821E
:1015C0008B8280910C028D831E822F83CE01019627
:1015D0009ECF483C510508F040C0882309F44DC017
:1015E000FE2CEE2009F406CF809109028D1127C050
:1015F000809108028C1123C090910E0290FD16C0BC
:10160000892F82958F70282F30E02115310571F0D8
:10161000F80196832F30310509F451CF8F5F982F51
:101620009295907F86818F70892B48CF87E0F80153
:10163000A8E0B2E001900D928A95E1F720C0C801C0
:101640000E946407811165CF80910E0281608093B2
:101650000E02C8010E940F0712C0682D9A8A898A5B
:10166000A6017A899E2D0E94710787E0F5011192EB
:101670008A95E9F72FCFF12C02C0FF24F3948F2D28
:101680006496ECE00C943321AEE0B0E0EAE4FBE0D9
:101690000C942121288739874A875B876C877D874F
:1016A0008E87CE0108960E94A009882369F06C8578
:1016B000662309F45FC0288539854A855B857D8569
:1016C0008E850E947B0756C087E0FE013896DE01BA
:1016D000119601900D928A95E1F76C85662309F4C5
:1016E00049C08091CF0190E09C012F5F3F4F277050
:1016F00033274091CE0150E02417350709F441C04B
:101700006D8367E070E00E94F320DC01A053BE4FC0
:1017100097E0FE01319601900D929A95E1F72093A2
:10172000CF010E94F40826C090E067E070E00E94BC
:10173000F32080539E4F0E94A009882379F1809165
:10174000CE0190E067E070E00E94F320FC01E053DE
:10175000FE4F208131814281538164817581868170
:101760000E947B078091CE0190E0019687709927B7
:101770008093CE018091CE019091CF018913D4CF77
:101780000DC00E9444071092CF011092CE01E8E0F4
:10179000F2E087E0DF011D928A95E9F72E96E2E0FC
:1017A0000C943D2180911702869586958695089523
:1017B000809117028770089590911702977081E0C9
:1017C00009F480E008958091230208959091230206
:1017D000892B809323020895809590912302892379
:1017E000809323020895109223020895909122027B
:1017F000892B80932202089580959091220289235B
:1018000080932202089510922202089508950E9462
:10181000060C08950E94070C089590911902292F33
:101820002823821729F0982B909319020E940A0C02
:10183000089590911902292F282331F0809589234A
:10184000809319020E940A0C08958091190288233E
:1018500029F01092190280E00E940A0C08950F935B
:101860001F93CF93DF930091000110910101C0916C
:10187000230280912202C82B80911902882331F023
:10188000C82B0E94AD1881110E94250CF801C0835D
:10189000C0910001D091010148E050E06FE072E09A
:1018A000CE010E944821892B59F088E0FE01AFE06B
:1018B000B2E001900D928A95E1F7CE010E9458188E
:1018C000DF91CF911F910F9108950E942F0C0895E1
:1018D0000E94060C08950E94680C089590911802C9
:1018E000292F282331F080958923809318020E94A4
:1018F0006B0C08950E94060C08959091530292FF7C
:1019000011C0982F990F990F990F692B60931702A7
:101910000E94BC07809117028695869586950E9445
:101920007A0C08950E94BC0708951092170280E077
:101930000E947A0C089590911702809589238093D4
:101940001702282F277069F4981759F090915302C5
:1019500092FF07C08695869586950E94C8070E94CB
:10196000950C08959091530292FB222720F9281795
:1019700069F080FB92F9909353028091520290910A
:1019800053020E94FB0C82E00E949B0C0895809100
:10199000530282FB882780F991E089270E94B20CCC
:1019A000089581E00E94B20C089580E00E94B20C7C
:1019B00008956FEF7FEF80E090E00E949A210895F4
:1019C00080E090E00E946621853E9E4F19F40E94BF
:1019D000F116089580E0089582E090E00E945E2173
:1019E000089583E090E00E945E21089584E090E0F5
:1019F0000E9466210895BC0184E090E00E949A2133
:101A00000895AB01BC018FE090E00E948E21089503
:101A1000AB01BC0183E190E00E948E21089560E05B
:101A200070E0CB010E94080D089560E070E0CB01EA
:101A30000E94010D0E940F0D0895A8E0B0E0E3E2BE
:101A4000FDE00C94212165EE7EEF80E090E00E94A5
:101A50009A2160E082E090E00E947C2181E0809306
:101A6000CD0161E083E090E00E947C2160E074E1C0
:101A700084E090E00E949A2160E086E090E00E947D
:101A80007C2160E087E090E00E947C2140E050E013
:101A9000BA0188E090E00E948E2160E083E290E04D
:101AA0000E947C2160E08CE090E00E947C2160E05C
:101AB0008DE090E00E947C2119821A821B821C8298
:101AC0001D821E821F82188648E050E067E170E0A8
:101AD000CE0101960E946C2140E050E0BA018FE1F6
:101AE00090E00E948E2180E00E940A170E943F171A
:101AF0000E94150D2896E2E00C943D210E941D0DD8
:101B00000895682F8EE090E00E947C210895A6E061
:101B1000B0E0EDE8FDE00C941F210E94BA198C01A1
:101B200080912402909125020817190781F01982EB
:101B30001A820E94BA19682F49815A81792F80E050
:101B400090E00E943C041093250200932402269604
:101B5000E4E00C943B210E94C61960933402709318
:101B6000350280933602909337026093300270936F
:101B700031028093320290933302089581E00895F8
:101B800081E008950E94C00D089508950E94C50D3A
:101B900008950E94C50D08950E94C90D08950E94E0
:101BA000C50D08950E94CF0D08950E94C50D08959A
:101BB00083EA90E10E940B120E94D50D0E94D20D83
:101BC00008950E94C60D0E94C50D08950E94E00C64
:101BD000811102C00E947E0D0E94EC0C809338029D
:101BE0000E94F60C90935302809352020E942E1290
:101BF0000E94F10C0E9492078091CC010E94A707DD
:101C000008950E94B1190E944F170E9463110E940B
:101C1000E60D0E9410040E94CC0D0895A6E0B0E0ED
:101C2000E4E1FEE00C9415210E94BE0D811103C079
:101C30000E94870D62C00E94791126E2E22E22E006
:101C4000F22E5701D12CF501019111915F018D2DDB
:101C50000E94A51080279127D394F5E0DF1619F094
:101C6000892B89F302C0892B19F38091380281FDF9
:101C70000E94AE100E94C20D782E10E0662463947C
:101C8000812F0E94A5104C01F701A080B180A826E9
:101C9000B926A114B10449F100E0CC24C394D12C9D
:101CA000C5018C219D21892BC1F07720B1F00983DA
:101CB0001A830E94BA199C838B836D8221E0C40130
:101CC0008C219D21892B09F420E049815A816B8167
:101CD0007C818D81922F0E943C040F5FCC0CDD1C17
:101CE0000F30F1F6F701918280821F5FF2E0EF0E74
:101CF000F11C153029F60E94AB0D0E942304269694
:101D0000EEE00C9431211F93CF93DF930E94B80F24
:101D1000EC01C11580E5D807E8F5C11590E4D907B5
:101D200008F0ACC0C03ED10530F5CD3CD10508F07F
:101D300098C0C83AD10578F4C53AD10508F087C0F3
:101D4000C130D10509F480C008F4F9C0C430D10510
:101D500008F0F8C0F4C0C33CD10508F0F0C0C85A80
:101D6000D0E0CC0FDD1FC75BDE4F0990D881C02DBE
:101D7000CE019464E8C0C11580E2D80708F0D2C053
:101D8000C11591E0D90708F06FC0C83ED10508F42D
:101D9000D9C0D5C0C03682E5D80738F5C03492E541
:101DA000D90708F07DC0C03282E5D80708F070C0BE
:101DB000C11592E5D90708F488C04C2F4695469581
:101DC00050E0F5E0440F551FFA95E1F7C37021E0AC
:101DD00030E0C90102C0880F991FCA95E2F7EA01F5
:101DE000C82BD92BCE019D68AEC0C03A82E5D8077A
:101DF000C8F48C2F8F71C03892E5D90708F080C0E5
:101E00008695869590E065E0880F991F6A95E1F7C1
:101E1000C37021E030E002C0220F331FCA95E2F701
:101E20003A686BC0C03C82E5D80708F470C0C03E79
:101E300092E5D90708F083C0CF71DD27DC2FCC27CE
:101E4000CE01806F906A7FC081E090E07CC0C55A6F
:101E5000D0E0C158DE4F8881C82FD0E0CE01906419
:101E600072C0CE0190656FC08D2F0E945410182F44
:101E7000CE0199270E94B80F1F715FC0CE0199272C
:101E80000E94B80FCC27DF70D06A8C2B9D2B5BC0D3
:101E9000CF71D0E0DC2FCC27CE01816F906A53C088
:101EA0008C2F8F718695869590E09C0175E0220FAE
:101EB000331F7A95E1F7C37081E090E002C0880F8C
:101EC000991FCA95E2F79C6818C08C2F8F710E94E9
:101ED000541095E0D695C7959A95E1F7CF70D0E06C
:101EE000DC2FCC27282F30E084FF05C084E0220FB0
:101EF000331F8A95E1F7D069CE01822B932B23C043
:101F000090E0D82FCC27CE01846F906A1CC08C2F14
:101F10008F710E9454108F7190E0D82FCC27CE0182
:101F2000906211C08D2F8F710E945410182FCE0116
:101F300099270E94B80F1F719062912B04C080E016
:101F400090E001C0CE01DF91CF911F9108957530CF
:101F500038F46F3028F4462F672F0E94E612089558
:101F600080E090E008950E94A70F0E94830E0895DC
:101F70008238910569F1B0F48133910509F475C097
:101F800048F48932910509F467C08A32910509F451
:101F900071C008958533910509F459C089339105BD
:101FA000B9F00895833E910589F138F4803E91059A
:101FB000D1F0823E910529F10895863E9105C9F13F
:101FC000873E9105D9F1843E910509F06CC027C088
:101FD0002091520220FD57C021FD55C0209153028F
:101FE00023FD5BC008958091520280FD48C080911E
:101FF000530280FF48C08091520284FD46C083EEA8
:1020000051C08091520282FF3CC0F5CF80915202B4
:1020100082FD37C08091530280FD35C0ECCF8091A6
:10202000530281FF36C08091520284FD2EC087EE9C
:1020300039C08091520283FF2AC0F5CF80915202AD
:1020400083FD25C08091530281FD23C0ECCF809198
:10205000520285FD22C01FC08091520285FD1BC027
:102060008091530283FF19C00AC08091520286FDFD
:1020700016C017C08091520286FD13C010C089E3BC
:1020800011C082EE0FC080EE0DC080E00BC086EE66
:1020900009C084EE07C085E305C089E203C08AE277
:1020A00001C081E390E008959091520292FF10C028
:1020B00041E0282F2471243009F040E031E0282F3E
:1020C0002871283009F030E0431711F02CE0822706
:1020D00093FF10C041E0282F2471243109F040E023
:1020E00031E0282F2871283109F030E0431711F032
:1020F0002CE082273091530230FF10C051E0282F8E
:102100002171213009F050E041E0282F287128305A
:1021100009F040E0541711F029E0822731FF10C088
:1021200041E0282F2171213109F040E031E0282FD2
:102130002871283109F030E0431711F029E0822797
:1021400094FD877E089580E00895E82FF0E0EE0F7B
:10215000FF1FE25AFD4F808191810895089580EA22
:102160008A95F1F7089500C008950E94AF10089570
:1021700008950E94B81008950E94B91008950E9411
:10218000B81008950E94BF100895F894E82FE295C2
:10219000EF70F0E031A1282F2F7081E090E001C0B6
:1021A000880F2A95EAF7982F9095932391A392A1EF
:1021B000892B82A3789408950F931F93CF93DF9375
:1021C000C1E9D1E089918F3F11F00E94C51081E0F3
:1021D000C639D807B9F7C2E8D1E001E911E0899121
:1021E0008F3F11F00E94C5100C171D07C1F7DF913A
:1021F000CF911F910F910895A0E0B0E0E2E0F1E1EE
:102200000C941A218C01C62FD0E0CE018F569E4F20
:102210006C01FC0190819F3F09F450C0B62EF894E8
:10222000E92FE295EF70F0E081A19F7021E030E0AE
:1022300001C0220F9A95EAF7822B81A382A12095F3
:10224000282322A378940E94B310E2E8F1E041E948
:1022500051E021E030E0E12CF12C61916F3F89F0F9
:10226000A62FA295AF70B0E090968C9190E06F7021
:1022700002C0959587956A95E2F780FD02C0C90175
:1022800002C080E090E0E82AF92A220F331F4E179F
:102290005F0719F7F60180818F3F11F00E94C5108A
:1022A00061E0E114F10409F460E08B2D0E94B510A7
:1022B000CC0FDD1FC00FD11FF982E882CDB7DEB78A
:1022C000E9E00C9436210E94DC108AE0EEE5F2E0B1
:1022D000DF01982F1D929A95E9F7E4E5F2E0DF011E
:1022E0001D928A95E9F785E00E94B4110E94C21000
:1022F0000895AAE0B0E0EFE7F1E10C941E218E0111
:102300000F5F1F4F8AE0F80111928A95E9F7F12CCF
:102310006F2DC8010E94FC10F394F5E0FF12F8CF76
:102320004AE050E0B80184E592E00E94482121E0B3
:10233000009709F420E0892B41F08AE0F801A4E538
:10234000B2E001900D928A95E1F745E06EE572E00A
:1023500084E592E00E94B511182F0E94BC10812FD5
:102360002A96E5E00C943A210895EF92FF920F939C
:102370001F93CF93DF937C018B01C42F222351F055
:1023800081E080933B020E94BA1990933A028093B5
:10239000390204C080913B02811102C080E01CC060
:1023A0008091390290913A020E94D2190597B0F3B8
:1023B000D0E0CC0FDD1FAE01B701C8010E9448215B
:1023C000892B39F0AE01B701C8010E94552181E087
:1023D00001C080E010923B02CDB7DEB7E6E00C947E
:1023E00039210E940E0E08950E9457190E94A61BC3
:1023F0000E94D80D0E94C01B0E94010E0E94CD1B9E
:102400000E94D21B0E94F1110E94EC1B0E94831AB1
:102410000E94E10DF5CF9093A7018093A601089546
:102420000E94D90C089580E00E94A5108170089543
:102430000E9479112FEF86E791E021508040904073
:10244000E1F700C000000E9479110E941312882356
:1024500021F00E9410120E94071A08950E9418127B
:10246000089584E00895E82F862F90E06EE170E0F3
:102470000E94F320242F30E0220F331F280F391F32
:102480008E2F90E066E970E00E94F320820F931F88
:10249000889608950F931F93CF93DF938430A0F411
:1024A000653090F44F3080F40E9433128C010E940A
:1024B0005E2190E0D82FCC27C80101960E945E21B2
:1024C0009E01282BC90102C080E090E0DF91CF91EE
:1024D0001F910F9108950F931F93CF93DF93843033
:1024E00080F4653070F44F3060F4E9010E943312DB
:1024F0008C016D2F0E947C216C2FC80101960E94D7
:102500007C21DF91CF911F910F9108951F93CF935D
:10251000DF93D0E0C0E010E0412F6C2F8D2F0E94A0
:10252000E6029C01412F6C2F8D2F0E946B121F5FC2
:102530001F3091F7CF5FC53071F7DF5FD43051F7AF
:10254000DF91CF911F910895EF92FF920F931F9308
:10255000CF93DF93EA017A01E60EF71E8C01C801E2
:102560008896CE15DF0569F0083522E0120720F4C1
:102570000E945E21888301C0188221960F5F1F4F41
:10258000EECFCDB7DEB7E6E00C943921EF92FF92A3
:102590000F931F93CF93DF93EA017A01E60EF71EA4
:1025A0008C01C8018896CE15DF0559F0083522E068
:1025B000120718F468810E947C2121960F5F1F4F3B
:1025C000F0CFCDB7DEB7E6E00C943921843038F493
:1025D000653028F44F3018F40E944A12089580E0C4
:1025E00090E0089580E1089580E891E00895EF92E9
:1025F000FF920F931F93CF93DF93EA017A01E60EC8
:10260000F71E8C01C80180589D4FCE15DF0569F07B
:10261000003821E0120720F40E945E21888301C067
:10262000188221960F5F1F4FEDCFCDB7DEB7E6E0E2
:102630000C943921EF92FF920F931F93CF93DF9366
:10264000EA017A01E60EF71E8C01C80180589D4F01
:10265000CE15DF0559F0003821E0120718F4688123
:102660000E947C2121960F5F1F4FEFCFCDB7DEB7C1
:10267000E6E00C943921CF93DF93C0E8D2E060E02C
:10268000CE010E947C212196C11584E0D807B9F7BC
:10269000DF91CF910895A8E0B0E0E1E5F3E10C947B
:1026A0001721F82E8FE08F1508F474C08FEF93E098
:1026B0000E945E2181116EC000E812E0FF2071F0DF
:1026C000011594E0190709F465C0C8010E945E2154
:1026D000811101C0FA940F5F1F4FF0CFFE013196B8
:1026E0006F0188E011928A95E9F77801FFEFEF1A00
:1026F000FF0AC8010E945E2189831A82882309F497
:1027000049C0813009F040C0580182E0A80EB11CD8
:10271000C7010E945E218A838823E1F19FEF980F11
:10272000933060F4780193E0E90EF11CC5010E943A
:102730005E218B83882371F11C8226C0843019F5B9
:102740004E01E3E08E0E911C02E010E07501FFEFF8
:10275000EF1AFF0AC5010E945E21F40181934F0127
:102760008823C1F08C3741F4E2E0F0E0EC0FFD1F6C
:10277000E00FF11F108208C00F5F1F4F5701073095
:10278000110521F707C0750160E0C6010E9494158C
:102790008701ABCF2896ECE00C943321CF93DF93E5
:1027A00086319C4709F5EB010E94E30B9D8199233B
:1027B00071F08A7A91E009F490E090933C028111E3
:1027C00002C089E201C085E30E94F71809C0809128
:1027D0003C02811102C089E201C085E30E94FF181A
:1027E0000E94650C80E001C081E0DF91CF910895E7
:1027F000CF93DF93FC01DB0115968C91882309F4BC
:10280000DDC09F0130572332310508F0D8C0EF01F9
:102810000E94F60C9093530280935202FE01E15005
:10282000F047E232F10520F4EA5BFF4F0C940421FB
:10283000809152028160AAC0809153028860B2C028
:10284000809152028260A2C08091520220C0809189
:10285000520288609BC0809153021EC08091530237
:102860008260A0C080915202806190C0809152022B
:1028700080628CC080915202806488C00E944407AC
:1028800080915202806882C0809152028860846088
:102890007DC0809153028260816084C08091520229
:1028A0008E7F74C080915302877F7CC080915202DA
:1028B0008D7F6CC08091520220C080915202877F30
:1028C00065C0809153021EC0809153028D7F6AC003
:1028D000809152028F7E5AC0809152028F7D56C0E5
:1028E000809152028F7B52C00E9444078091520215
:1028F0008F774CC080915202877F8B7F47C0809139
:1029000053028D7F8E7F4EC08091520282FB222720
:1029100020F991E0922790FB82F990FB83F936C071
:1029200080915302982F909591708E7F892B90FB08
:1029300081F938C08091520286FB222720F991E06C
:10294000922790FB86F922C00E9444078091520290
:1029500087FB222720F991E0922790FB87F916C088
:1029600081E001C080E00E94810D1EC08091520272
:1029700084FB222720F991E0922790FB84F906C07E
:1029800080915202982F909590FB80F9809352028B
:102990000BC08091530283FB222720F991E09227FC
:1029A00090FB83F9809353028091520290915302DD
:1029B0000E94FB0C0E94440780E001C081E0DF918F
:1029C000CF9108958F929F92BF92CF92DF92EF9214
:1029D000FF920F931F93CF93DF93E82FF0E0E0591E
:1029E000FC4FB490282F26952695269530E0F901C6
:1029F000E05FFB4FE4908770F12C082E02C0F59445
:102A0000E7940A94E2F791E0E922FF24F901E0500B
:102A1000FC4FC490D12C082E02C0D594C7940A94C0
:102A2000E2F7E1E0CE22DD24F901E051FC4FC49150
:102A3000D0E002C0D595C7958A95E2F7C170DD2731
:102A4000062F10E0E114F10471F081EE0E94780489
:102A5000C801009741F0EFE9FFE03197F1F700C0BE
:102A600000000197F6CFC114D10439F44801B80130
:102A70008B2D0E94E204C8010EC086EE0E947804ED
:102A8000C801009799F3EFE9FFE03197F1F700C033
:102A900000000197F6CF009741F0EFE9FFE0319792
:102AA000F1F700C000000197F6CFCD2819F5EF2807
:102AB00079F081EE0E94B8040115110549F08FE903
:102AC0009FE00197F1F700C0000001501109F4CF19
:102AD000CD2BF1F08CE20E94FA0481149104C1F034
:102AE000EFE9FFE03197F1F700C00000F1E08F1A45
:102AF0009108F3CF86EE0E94B804C8010097B9F29E
:102B0000EFE9FFE03197F1F700C000000197F6CF41
:102B1000DF91CF911F910F91FF90EF90DF90CF90B9
:102B2000BF909F908F900895EF92FF921F93CF9345
:102B3000DF93EC01162F8881882309F455C081307A
:102B400009F04DC08981813041F47E0182E0E80EB8
:102B5000F11C8A810E94FA0409C0823049F47E0186
:102B6000E2E0EE0EF11C8A810E947804E7012BC09E
:102B7000833041F47E01F2E0EF0EF11C8A810E9465
:102B8000B804F4CF843011F021961DC02A8122961A
:102B900080E090E030E0205331092A30310548F4DC
:102BA0006AE070E00E94F320820F931F2196288133
:102BB000F1CF009741F0EFE9FFE03197F1F700C066
:102BC00000000197F6CF812F90E0009759F0EFE9D0
:102BD000FFE03197F1F700C000000197F6CF612FB9
:102BE0000E94E2142196A7CFDF91CF911F91FF9011
:102BF000EF9008950F931F93CF93DF93C42FD22F9D
:102C0000FC0185818823B1F040933F020E94BA19EC
:102C100090933E0280933D0280E28C0F883008F052
:102C20004DC0C77081E001C0880FCA95EAF70E94C5
:102C3000040544C080913F02481330C080913D029A
:102C400090913E020E94D219883C910538F510E21D
:102C50001D0FCD17B9F080E28C0F883040F4C7709B
:102C600081E001C0880FCA95EAF70E940B05183071
:102C700010F581E09D2F977001C0880F9A95EAF7B3
:102C80000E940405802F0E94FA041830B8F4D7700F
:102C900081E001C0880FDA95EAF70AC080E28C0F64
:102CA000883060F4C77081E001C0880FCA95EAF7E8
:102CB0000E940B0503C0802F0E94FA04DF91CF9180
:102CC0001F910F9108950F93FC01E851FC47E730E5
:102CD000F10590F5CB01E859FF4F0C94042106E271
:102CE00021EE41EE6AE17CE723C007E225EE45EEE6
:102CF0006BE17CE71DC006E221EE40EE68E17CE777
:102D000017C007E225EE44EE69E17CE711C006E258
:102D100021EE42EE6CE17CE70BC007E225EE46EEC9
:102D20006DE17CE705C008E221E045EE6EE17CE75D
:102D30000E94FA1580E008C0FB018581882319F004
:102D400010923F0201C081E00F9108951F93CF932D
:102D5000DF9387372CE7920721F088379C4759F09B
:102D600031C0FB01C581CC2319F00E94E81609C0CF
:102D70000E94E81618C0FB01C581CC2391F00E9487
:102D8000EB160E94BC070E94EE16D82F0E94EB168D
:102D9000C82F0E94E8164D2F6C2F0E94EA08C0E051
:102DA00012C00E94EB160E94C8070E94EE16182F50
:102DB0000E94EB16D82F0E94E816412F6D2F0E941B
:102DC000EA0801C0C1E08C2FDF91CF911F910895D7
:102DD000809104010895809103010895809102017A
:102DE000089584E290E00E945E21843281F485E2BD
:102DF00090E00E945E21883051F486E290E00E94CB
:102E00005E2191E0873109F090E0892F01C080E0D8
:102E100081700895CF93C82F811102C06FEF01C058
:102E200064E284E290E00E947C21C11102C06FEF55
:102E300001C068E085E290E00E947C21C11102C0DF
:102E40006FEF01C067E186E290E00E947C21CF91A4
:102E50000895089587E290E00E945E21682F70E057
:102E600080E090E008950895CF93C62F0E94331715
:102E70006C2F87E290E00E947C21CF91089580E042
:102E80000E940A1760E070E0CB010E9434170E9494
:102E900086120E943B1381E00E940A1708950E9447
:102EA00029170E942A170E9433170E94F1168111D8
:102EB00002C00E943F17089508959C01FB0185817F
:102EC000882351F0A90157574038510530F4C90102
:102ED0000E944B1380E0089581E008952FEFFC01DC
:102EE000208308950E946E17089580E00895A0E061
:102EF000B0E0EDE7F7E10C941921EC01D62E0E9429
:102F000075178111BEC0E8818E2F90E0FC013197CA
:102F1000E331F10508F0AFC0E159FF4F0C940421F3
:102F200019828CE06BC08981823089F030F4813065
:102F300009F0A1C00E94C6190CC0833079F084301A
:102F400009F099C01A821B821C821D8296C00E94C1
:102F50002A179A838B837C836D838FC0CA807E01FE
:102F600000E010E0AC2CB12CC501800F911F05973B
:102F700008F083C08C2D800F0E94A510F701938369
:102F800084830F5F1F4FF2E0EF0EF11C0E3011052E
:102F900059F773C08981823039F0853009F06BC0F0
:102FA0008A810E945C1769C06A817B818C819D81C6
:102FB0000E940A210E94341760C04B816A81898176
:102FC0000E944A129C838D8358C02C813D813227F8
:102FD000232732274B816A8189810E946B124DC061
:102FE0000E9486124AC06D2DCE010E94721745C004
:102FF0000E94F21224C00E94F41299838A833DC079
:103000006B8170E089819A81AE014C5F5F4F982798
:10301000892798270E94F71230C06B8170E0898160
:103020009A81AE014C5F5F4F9827892798270E94AD
:103030001A1323C00E943B1320C00E9431128983BF
:103040001CC06B8170E089819A81AE014C5F5F4F3B
:103050009827892798270E94A4120FC06B8170E0DF
:1030600089819A81AE014C5F5F4F98278927982705
:103070000E94C61202C08FEF88836D2DCE010E9480
:103080007A1ACDB7DEB7EAE00C9435219093450269
:10309000809344020895E0914402F09145023097F4
:1030A00029F00190F081E02D0995089580E00895C0
:1030B000E0914402F0914502309721F00280F381C3
:1030C000E02D09950895A3E0B0E0E9E6F8E10C945D
:1030D0002121209142023091430228173907A1F0A3
:1030E0009093430280934202E0914402F0914502A2
:1030F000309751F023E029839B838A830084F185F4
:10310000E02DCE01019609952396E2E00C943D2135
:10311000A3E0B0E0EEE8F8E10C9421212091400218
:103120003091410228173907A1F090934102809312
:103130004002E0914402F0914502309751F024E0C2
:1031400029839B838A830084F185E02DCE0101963B
:1031500009952396E2E00C943D21E0910001F09165
:103160000101329697E080E0915029F021912223CD
:10317000D9F38F5FF9CF0895882371F02091000172
:1031800030910101F9013296285F3F4F91918917E3
:1031900029F0E217F307D1F780E0089581E0089560
:1031A0009C01FC0132969FEF80E04191461789F027
:1031B0009F3F19F4411101C0982F8F5F8630A9F706
:1031C0009F3F39F0F901E90FF11D97FDFA956283F0
:1031D000089508959C012A5F3F4FFC0142814613E8
:1031E00001C01282019682179307B9F70895682FDC
:1031F00080910001909101010E94D0180895682FDC
:1032000080910001909101010E94EA180895E091D7
:103210000001F0910101329686E0DF011D928A954E
:10322000E9F7089508950E941219089583E08093A4
:1032300046020E9413190895811102C081E001C065
:1032400082E0809346020E94131908950E941C197F
:10325000089581E0809346020E94131908950E9408
:103260002919089508950E94321908950E9433196A
:1032700008950E94321908950E94321908950E94FB
:1032800032190895CF930E943C190E9479110E942F
:103290003919C0E08C2F0E94A510892B29F4CF5F2B
:1032A000C530C1F780E001C081E0CF910895089555
:1032B0001F920F920FB60F9211248F939F93AF938B
:1032C000BF9380914702811113C080916802909151
:1032D0006902A0916A02B0916B024196A11DB11DD5
:1032E0008093680290936902A0936A02B0936B0284
:1032F000BF91AF919F918F910F900FBE0F901F9034
:10330000189580917002843031F10E94F30310927D
:10331000470220E488E190E00FB6F894A8958093E6
:1033200060000FBE2093600083B7817F846083BFFD
:1033300083B7816083BF7894889583B78E7F83BF7E
:103340000FB6F894A8958091600088618093600022
:10335000109260000FBE08950E9444070E94F80377
:10336000089582E084BD93E095BD9AEF97BD809368
:103370006E0008952FB7F8948091680290916902C9
:10338000A0916A02B0916B022FBF08952FB7F894F5
:10339000609168027091690280916A0290916B025B
:1033A0002FBF08959C014FB7F894809168029091C7
:1033B0006902A0916A02B0916B024FBF821B930B0E
:1033C000089578941F920F920FB60F9211248F9345
:1033D0009F93AF93BF938091680290916902A091EF
:1033E0006A02B0916B020196A11DB11D8093680223
:1033F00090936902A0936A02B0936B02BF91AF9160
:103400009F918F910F900FBE0F901F90189581E0A4
:103410008093E00080E28093D8001092C9008FE191
:103420009EE40197F1F700C0000087E090EBDC011B
:103430008093790290937A02A0937B02B0937C02EE
:103440009CE088E10FB6F894A895809360000FBEC9
:1034500090936000FFCF9CE088E10FB6F894A895A8
:10346000809360000FBE90936000FFCF8091500268
:103470000895089508959B01909170029430F1F49D
:103480008F708093E9008FEF9091E800815095FD57
:1034900006C095ED9A95F1F700008111F5CF809166
:1034A000E80085FF0BC0BA01C90140E050E00E946E
:1034B000611C8091E8008E778093E800089543E0D6
:1034C00050E0BC0184E00E943B1A0895CF93DF9343
:1034D000EC0148E050E0BC0181E00E943B1A88E02A
:1034E000FE01A8E4B2E001900D928A95E1F7DF9128
:1034F000CF910895603231F4BC0140E250E082E0A7
:103500000E943B1A0895A0E2B0E0E9E8FAE10C94C9
:10351000212180917002843011F583E08093E900CD
:103520008091E80082FF1BC08091E80085FF0AC0FF
:1035300040E050E060E270E0CE0101960E94A61CDF
:1035400091E001C090E08091E8008B778093E800E3
:10355000992329F060E2CE0101960E947717A09688
:10356000E2E00C943D210E942F19089560916C02B5
:1035700081E0611101C080E00E94161908959091C8
:10358000700281E0943009F080E060916C020E944A
:103590001C19089542E061EC81E00E94A41D42E202
:1035A00061EC84E00E94A41D42E261EC82E00E9492
:1035B000A41D42E260EC83E00E94A41D9091700281
:1035C00081E0943009F080E060916C020E9426193D
:1035D000089580917202833009F45FC030F4813025
:1035E00071F0823009F499C008958A3009F485C0D9
:1035F0008B3009F46AC0893009F0A7C020C08091DF
:103600007102813A09F0A1C08091E800877F809320
:10361000E8008091750290917602892B21F468E090
:1036200088E492E003C060E080E090E070E00E94F7
:10363000EB1C8091E8008B778093E80008958091DF
:103640007102813209F081C08091750290917602F9
:10365000009719F0029709F078C08091E800877F01
:103660008093E8008091E80082FD05C0809170029F
:103670008111F8CF6AC08091F200823031F48091DC
:10368000F100813011F0863021F48091F1008093B7
:1036900050028091E8008B7754C080917102813A8A
:1036A00009F053C08091750290917602892B09F040
:1036B0004CC08091E800877F8093E8008091E8000B
:1036C00080FFFCCF80910F0137C080917102813261
:1036D000E1F58091750290917602892BB1F5809188
:1036E000E800877F8093E8000E94D91D80917302D3
:1036F00080930F010E9444070895809171028132E6
:1037000021F58091E800877F8093E8000E94D91D11
:103710008091740280935102089580917102813AE0
:10372000A1F48091E800877F8093E8008091E80011
:1037300080FFFCCF809151028093F1008091E800DE
:103740008E778093E8000E94D91D089584B7877F03
:1037500084BF0FB6F894A89580916000886180932B
:103760006000109260000FBE90E080E80FB6F89401
:1037700080936100909361000FBE0E942919089503
:103780000E942B1E0E947E1EE2EEF0E0808184608B
:10379000808378940E94D820089585E091E00E946B
:1037A00046180895809170028530A9F480917002C6
:1037B000853079F40E94811980916E028823B1F3DB
:1037C0000E944219882391F30E944B1C0E944407D7
:1037D000EDCF0E94AC19089508959A0140917702A7
:1037E000509178020E94F51B0895492F55274330C8
:1037F0005105C9F060F44130510581F04230510566
:1038000009F041C08BE590E042E554E040C0413210
:103810005105E1F04232510531F135C082E190E0CD
:103820004DEA54E034C099278130910549F028F0E1
:10383000029749F5E0E2F4E005C0EEE4F4E002C0EE
:10384000EEE3F4E0849190E0AF0121C063307105B4
:10385000D0F4660F771FFB01E156FE4F4081518186
:1038600089E090E014C06330710568F4FB01EE0F4D
:10387000FF1FE756FE4F40815181FB01EA56FE4F84
:10388000808190E004C080E090E040E050E0F901E9
:1038900051834083089584E089BD86E089BD09B4E1
:1038A00000FEFDCF8091D8008F7D8093D80080915D
:1038B000E00082608093E0008091E00081FDFCCF19
:1038C0000895A0E0B0E0E7E6FCE10C941B21EC01D8
:1038D0008B017A010E94F81D811133C0E114F104BB
:1038E00039F0F70180819181081B190BC80FD91F8E
:1038F000C12CD12C0115110519F18091E80085FD2D
:1039000016C08091E8008E778093E800E114F104FE
:1039100049F0F70180819181C80ED91ED182C08201
:1039200085E00FC00E94F81D882321F30AC0899109
:103930008093F10001501109FFEFCF1ADF0ADACFAF
:1039400080E0CDB7DEB7E8E00C943721A0E0B0E02E
:10395000ECEAFCE10C941B21EC018B017A010E9442
:10396000F81D811133C0E114F10439F0F7018081B1
:103970009181081B190BC80FD91FC12CD12C01151F
:10398000110519F18091E80085FD16C08091E800CD
:103990008B778093E800E114F10449F0F70180810E
:1039A0009181C80ED91ED182C08285E00FC00E94CD
:1039B000F81D882321F30AC08091F10089930150FA
:1039C0001109FFEFCF1ADF0ADACF80E0CDB7DEB7FB
:1039D000E8E00C9437212091770230917802261785
:1039E000370748F06115710539F42091E8002E770A
:1039F0002093E80001C0B901FC0120E061157105C8
:103A000061F1809170028823D9F18530D9F18091DC
:103A1000E80083FD39C08091E80082FD2BC08091D1
:103A2000E80080FFEBCF8091F20090E06115710516
:103A300051F08830910538F421912093F1006150C4
:103A400071090196F3CF21E0089709F020E08091F9
:103A5000E8008E778093E800D1CF2111D2CF0AC041
:103A600080917002882361F0853061F08091E800D8
:103A700083FD0AC08091E80082FFF2CF80E00895C4
:103A800082E0089583E0089581E00895209177020F
:103A9000309178022617370748F06115710539F41F
:103AA0002091E8002E772093E80001C0B901FC01C5
:103AB00020E06115710579F180917002882309F485
:103AC0003DC0853009F43CC08091E80083FD3AC0D8
:103AD0008091E80082FD2CC08091E80080FFE9CF52
:103AE0008091F20090E06115710559F088309105E0
:103AF00040F424912093F1003196615071090196B0
:103B0000F2CF21E0089709F020E08091E8008E775D
:103B10008093E800CECF2111CFCF0AC080917002F0
:103B2000882361F0853061F08091E80083FD0AC050
:103B30008091E80082FFF2CF80E0089582E008954E
:103B400083E0089581E00895982F953068F590936B
:103B5000E900981739F07091EC002091ED00509138
:103B6000F00003C0242F762F50E021FD02C09F5F9C
:103B7000ECCF3091EB003E7F3093EB003091ED00C5
:103B80003D7F3093ED003091EB0031603093EB00DE
:103B90007093EC002093ED005093F0002091EE0024
:103BA00027FDE5CF80E008958F708093E90081E0E4
:103BB00008958091710287FF11C08091E80082FD15
:103BC00005C0809170028111F8CF11C08091E8008A
:103BD0008B770BC080917002882349F08091E800B8
:103BE00080FFF8CF8091E8008E778093E8000895F9
:103BF0002091E4003091E50095E64091EC00842F9F
:103C0000817040FF23C08091E80080FD1DC080913D
:103C10007002882399F0853099F08091EB0085FD42
:103C200011C04091E4005091E5002417350729F3B5
:103C3000915011F09A01E1CF84E0089582E0089557
:103C400083E0089581E0089580E008954091E800C0
:103C500042FFDDCF08950E94891E0E948C1EE0EE77
:103C6000F0E0808181608083E8EDF0E080818F77F3
:103C7000808319BCE3E6F0E080818160808310924C
:103C80006F0208950E94891E0E948C1E8091D800A8
:103C90008F778093D8008091D80080688093D80077
:103CA0008091D8008F7D8093D80084E089BD86E024
:103CB00089BD09B400FEFDCF1092700210926C0213
:103CC00010926E0210926D0242E060E080E00E946D
:103CD000A41D8091E1008E7F8093E1008091E2003D
:103CE00081608093E2008091E20088608093E2002E
:103CF0008091E0008E7F8093E0000895E3E6F0E09D
:103D000080818E7F808381E080936F020E94421EBB
:103D100008951092E20008951092E10008951F9214
:103D20000F920FB60F9211242F933F934F935F93EF
:103D30006F937F938F939F93AF93BF93EF93FF9373
:103D40008091E10082FF0BC08091E20082FF07C0FA
:103D50008091E1008B7F8093E1000E94D7208091C9
:103D6000E10080FF19C08091E20080FF15C08091C2
:103D7000E2008E7F8093E2008091E2008061809378
:103D8000E2008091D80080628093D80019BC85E061
:103D9000809370020E94B61A8091E10084FF30C0C7
:103DA0008091E20084FF2CC084E089BD86E089BD5B
:103DB00009B400FEFDCF8091D8008F7D8093D8009C
:103DC0008091E1008F7E8093E1008091E2008F7E00
:103DD0008093E2008091E20081608093E200809114
:103DE0006C02882311F084E007C08091E30087FD16
:103DF00002C081E001C083E0809370020E94BF1A7C
:103E00008091E10083FF29C08091E20083FF25C0FB
:103E10008091E100877F8093E10082E080937002CF
:103E200010926C028091E1008E7F8093E10080917E
:103E3000E2008E7F8093E2008091E20080618093B7
:103E4000E20042E060E080E00E94A41D8091F0006A
:103E500088608093F0000E94B31AFF91EF91BF91A8
:103E6000AF919F918F917F916F915F914F913F9112
:103E70002F910F900FBE0F901F9018951F920F92C9
